:020000040000FA
:060000000CEF08F01200F5
:060800000CEF08F01200ED
:06082A0001004C1000006B
:08083000600000002000000040
:08083800D9CFE6FFE1CFD9FFA3
:10084000040EE126DE6ADE6ADE6ADD6ADD52DD5212
:10085000FD0EDBCF14F0FE0EDBCF15F0166A176A23
:1008600015AE02D016681768D9CFE9FFDACFEAFFD4
:10087000030EEB501718E8AE02D0173408D014500E
:10088000EE5C1550EE581650EE581750EE580FE229
:100890000C0EE66EECEC07F0E552D9CFE9FFDACFAB
:1008A000EAFFEE2A000EEE22EE22EE22D1D7040E4F
:1008B000E15C02E2E16AE552E16EE552E7CFD9FF81
:1008C00012000F0EC16E070EB46E936A300E926E58
:1008D0000F0E946EF19E816A80901200D9CFE6FFD0
:1008E000E1CFD9FF020EE1268250020B01E0010E9A
:1008F000080DF3CF16F08250010B040DF3CF15F065
:100900008050200B01E0010EE824146E8050100B83
:1009100001E0010E142415241624DE6EDD6ADECFFC
:1009200014F0DDCF15F014C0F3FF15C0F4FF020E74
:10093000E15C03E200D0E16AE552E16EE552E7CF07
:10094000D9FF12008092320EE66E1AEC08F0E552E2
:100950008084320EE66E1AEC08F0E5528094320E76
:10096000E66E1AEC08F0E55212008082320EE66E56
:100970001AEC08F0E5528084320EE66E1AEC08F0AC
:10098000E5528094320EE66E1AEC08F0E552120041
:10099000380E816ED7DF320EE66EE66A4DDFE55225
:1009A000E552010E816ECEDF320EE66EE66A44DF5E
:1009B000E552E5520D0E816EC5DF320EE66EE66A37
:1009C0003BDFE552E552060E816EBCDF320EE66E6D
:1009D000E66A32DFE552E5521200010E816EB2DFA7
:1009E0000A0EE66EE66A28DFE552E5521200D9CF1C
:1009F000E6FFE1CFD9FF020E816EA4DF0A0EE66E9C
:100A0000E66A1ADFE552E552FD0EDBCFE6FFFE0E89
:100A1000DB50280DF350E552E724E76EFE0EE7CFDA
:100A2000DBFFFD0EDB6AFE0EDB50F36EFD0EDBCF4F
:100A3000F4FFF350F45C0BE2140E816E83DF320E90
:100A4000E66E1AEC08F0E552FD0EDB2AECD7E55213
:100A5000E7CFD9FF1200D9CFE6FFE1CFD9FFFE0ED5
:100A6000DB50816E82DF320EE66E1AEC08F0E55242
:100A7000E552E7CFD9FF1200D9CFE6FFE1CFD9FF8A
:100A8000FD0EDBCFE9FFFE0EDBCFEAFFEF500EE0FD
:100A9000FD0EDBCFE9FFDB2AFE0EDBCFEAFF01E331
:100AA000DB2AEF50E66ED7DFE552EAD7E552E7CF13
:100AB000D9FF12000201046B300E926EF00E936E9D
:100AC000EF0E006F00C281FF040E016F015100089C
:100AD00021E20051FE0BE842006F00C281FF050ECB
:100AE000E66EE66AA9DEE552E5528150100B09E098
:100AF0008150200B06E08150400B03E08150800BB9
:100B000001E10AD80201040502E1055104D0010502
:100B1000016FDCD7CFD71200F00E936E81CF03F2B6
:100B200002010315026F0F0E0015006F0051021134
:100B3000006F81CF03F2F00E0315026FF00E025D1D
:100B400001E0F7D7936A06D806C205F20201010E4A
:100B5000046F12000201076B100E075D14E20751CB
:100B6000EA6A600FE96E000EEA22EF50005D08E1CC
:100B70000751EA6A700FE96E000EEA22EFCF06F223
:100B80000729076FE9D706C281FF640EE66EE66AA1
:100B900053DEE552E55212000201086B070E085DB4
:100BA0001DE288DF0201096F0851EA6A0A0FE96E47
:100BB000020EEA2209C2EFFF0851EA6A0A0FE96E43
:100BC000020EEA22EF50460802E108D004D009C222
:100BD000E6FF41DFE5520201082BE0D70851EA6A3F
:100BE0000A0FE96E020EEA22EF6A12000201086B98
:100BF000070E085D16E20851EA6A0A0FE96E020E56
:100C0000EA22EF50E66E27DFE55202010829EA6A80
:100C10000A0FE96E020EEA22EF5001E102D0082B22
:100C2000E7D71200D9CFE6FFE1CFD9FFE652F25065
:100C3000800B01E0010EDF6EF29EA69EA69CA684AC
:100C4000FE0EDB50A96EFD0EDB50A86E550EA76E92
:100C5000AA0EA76EA682A6B2FED7A694DF50E8B071
:100C6000F28EE8A0F29EE552E552E7CFD9FF1200DE
:100C7000D9CFE6FFE1CFD9FFA69CA69EFE0EDB50A2
:100C8000A96EA680A85000D0E552E7CFD9FF120088
:100C900018DE7EDEA2DE3E0EE66EDDDEE552E66AA0
:100CA000010EE66EA4DEE552E5520201276B286BC9
:100CB000080E28AF02D0D89003D0275D000E285927
:100CC00047E2F8DEE66E27C2E9FF28C2EAFFD890C5
:100CD000E936EA36130EE926020EEA22E552E7501B
:100CE000EE6EED6A27C2E9FF28C2EAFFD890E93626
:100CF000EA36130EE926020EEA22EF50E66EABDE6C
:100D0000E55227C2E9FF28C2EAFFD890E936EA3661
:100D1000130EE926020EEA22EECF14F0EFCF15F003
:100D2000300E145E000E155A27C2E9FF28C2EAFFF2
:100D3000D890E936EA36130EE926020EEA2214C0EC
:100D4000EEFF15C0EDFF0201272B000E2823B0D7C0
:100D500015C218F016C219F0D89018361936D89066
:100D600018361936080E086E096A13C20DF014C23F
:100D70000EF0BFEC07F006501824166E075019202D
:100D8000176E020E086E096A17C20DF018C20EF037
:100D9000BFEC07F016500624146E17500720156E8E
:100DA000145002011925236F15501A21246F1DC2FA
:100DB00018F01EC219F0D89018361936D890183687
:100DC0001936080E086E096A1BC20DF01CC20EF01F
:100DD000BFEC07F006501824166E07501920176E46
:100DE000020E086E096A1FC20DF020C20EF0BFECA1
:100DF00007F016500624146E17500720156E145075
:100E000002012125256F15502221266F23C2E6FFFE
:100E100024C2E6FF20D8E552E552F3CF23F2F4CF07
:100E200024F225C2E6FF26C2E6FF15D8E552E552B8
:100E3000F3CF25F2F4CF26F2E66AE66AD8DDE55272
:100E4000E55223C2E6FF07DEE55225C2E6FF03DED8
:100E5000E552FFD71200D9CFE6FFE1CFD9FFFD0E53
:100E6000DBCF14F0FE0EDBCF15F0153404E2145086
:100E70000908000E155413E2370EE76EFD0EDBCFA6
:100E800014F0FE0EDBCF15F0E7501426000E1522ED
:100E9000FD0E14C0DBFFFE0E15C0DBFF12D0300EBE
:100EA000E76EFD0EDBCF14F0FE0EDBCF15F0E75042
:100EB0001426000E1522FD0E14C0DBFFFE0E15C019
:100EC000DBFFFD0EDBCF14F0FE0EDBCF15F014C000
:100ED000F3FF15C0F4FF00D0E552E7CFD9FF1200B1
:100EE0002A0EF66E080EF76E000EF86E020109006B
:100EF000F5502E6F0900F5502F6F03E12E6701D0DA
:100F00003DD00900F550296F0900F5502A6F0900FE
:100F1000F5502B6F09000900F550E96E0900F550F6
:100F2000EA6E090009000900F5502C6F0900F55020
:100F30002D6F09000900F6CF30F2F7CF31F2F8CF6C
:100F400032F229C2F6FF2AC2F7FF2BC2F8FF0201D4
:100F50002C5302E12D5307E00900F550EE6E2C07EB
:100F6000F8E22D07F9D730C2F6FF31C2F7FF32C2DF
:0E0F7000F8FF02012E07000E2F5BBFD7120004
:020F7E0009C0A8
:100F800013F008C012F008500D02F4CF07F0F3CFB1
:100F900006F009500E02F4CF09F0F3CF08F00D026D
:100FA000F3500726F4500822E86A092212500E0274
:100FB000F3500726F4500822E86A09220EAEE5EF46
:100FC00007F01250085E1350095A13AE000C0D5072
:080FD000085E0E50095A000CE6
:080FD800FF0EE3501A6E480EF3
:100FE00001D04C0EE76EE72EFED7E76AE72EFED75C
:080FF0001A2EF7D700001200D1
:080FF800000EF36E00EE00F0A4
:10100000080E01D81200EA6002D0EE6AFCD7F35055
:08101000E9601200EE6AFCD752
:0810180012EE40F022EE40F060
:10102000F86A019C70EC07F025EC08F048EC06F03B
:04103000FBD71200D8
:0C103400FF0EE350E84E1200000000D058
:0A10400000D000D0E82EFAD712000D
:02104A00120092
:04104C00EEEDEBE7F3
:10105000DEDDDBD7BEBDBBB77E7D7B773031323383
:0C106000343536373839414243444546A8
:00000001FF
